:100000000C9447000C9464000C9464000C946400FD
:100010000C9464000C9464000C9464000C946400D0
:100020000C9466000C9464000C9464000C946400BE
:100030000C9464000C9464000C9464000C946400B0
:100040000C9464000C9464000C9464000C946400A0
:100050000C9464000C9464000C9464000C94640090
:100060000C9464000C9464000C9464000C94640080
:100070000C9464000C9464000C9464000C94640070
:100080000C9464000C9464000C9464000A03112422
:100090001FBECFEFD0E4DEBFCDBF21E0A0E0B1E0D6
:1000A00001C01D92A231B207E1F710E0C7E4D0E031
:1000B00004C02197FE010E943103C634D107C9F75D
:1000C0000E94F4020C943A030C9400001F920F92C9
:1000D0000FB60F92112491E085B1892785B92FEFD2
:1000E00034E38CE0215030408040E1F700C0000054
:1000F000F3CF81E191E00E94B40060E08EE091E0F6
:100100000E94F7006FEF8EE091E00E94180160E01E
:100110008BE091E00E94F7006FEF8BE091E00E948E
:1001200018016FEF88E091E00E94180181E091E0F2
:100130000E94ED0180E091E00C94DA02CF9380E020
:1001400091E00E94ED0280E091E00E94ED02C82F54
:100150006FEF80E091E00E94E6026C2F80E091E07A
:10016000CF910C94E602089584B1806B84B92698EF
:100170008AB18C618AB980E58CBD81E08DBD8BB17F
:10018000837E8BB95A9A5B9A5C9A08958BB1837E71
:100190008BB98BB160FD10C090E0892B8BB98BB10E
:1001A00061FD10C090E0892B8BB98BB162FD10C04E
:1001B00090E0892B8BB9089594E0892B8BB98BB192
:1001C00061FFF0CF98E0892B8BB98BB162FFF0CF44
:1001D00090E1892B8BB908956EBD0DB407FEFDCF5C
:1001E0008EB50895FC0171836083428308951F9347
:1001F000CF93DF93EC01162F6A81888199810E9449
:10020000C60060E4888199810E94EC0060E08881EA
:1002100099810E94EC00612F888199810E94EC00F5
:1002200067E088819981DF91CF911F910C94C6007E
:100230001F93CF93DF93EC01162F6A8188819981F8
:100240000E94C60060E4888199810E94EC0061E010
:10025000888199810E94EC00612F888199810E9498
:10026000EC0067E088819981DF91CF911F910C9418
:10027000C6001F93CF93DF93EC01162F6A8188810C
:1002800099810E94C60060E4888199810E94EC00F7
:1002900062E1888199810E94EC00612F88819981B7
:1002A0000E94EC0067E088819981DF91CF911F91D6
:1002B0000C94C6001F93CF93DF93EC01162F6A8135
:1002C000888199810E94C60060E4888199810E949A
:1002D000EC0063E1888199810E94EC00612F8881A4
:1002E00099810E94EC0067E088819981DF91CF912C
:1002F0001F910C94C6001F93CF93DF93EC016A818A
:10030000888199810E94C60061E4888199810E9458
:10031000EC0062E1888199810E94EC0060E08881B4
:1003200099810E94EC00182F67E0888199810E94D2
:10033000C600812FDF91CF911F9108951F93CF9316
:10034000DF93EC016A81888199810E94C60061E493
:10035000888199810E94EC0063E1888199810E94E3
:10036000EC0060E0888199810E94EC00182F67E022
:10037000888199810E94C600812FDF91CF911F91C2
:100380000895FC01428308950F931F93CF93DF9349
:10039000EC018B016A81888199810E94C600B801B5
:1003A0000024660F771F001C660F771F001C672F45
:1003B000702D888199810E94EC00602F660F660F76
:1003C000888199810E94EC0067E088819981DF91A2
:1003D000CF911F910F910C94C60010927C0087E87A
:1003E00080937A00089580917C00807E682B6093D2
:1003F0007C0080917A00806480937A0083EA91E0A7
:100400000197F1F700C0000080917A0086FDFCCFD3
:10041000809178009091790008950F931F93CF9366
:10042000DF9361E08EE091E00E943901C1E0D0E00D
:1004300001E010E02FEF84E39CE0215080409040E9
:10044000E1F700C00000B8010C2E01C0660F0A944D
:10045000EAF78EE091E00E9439012196C930D1057A
:1004600049F7DF91CF911F910F9108950F931F933B
:10047000CF93DF9361E08BE091E00E943901C1E00E
:10048000D0E001E010E02FEF84E39CE021508040B9
:100490009040E1F700C00000B8010C2E01C0660FCB
:1004A0000A94EAF78BE091E00E9439012196C93065
:1004B000D10549F7DF91CF911F910F910895CF9307
:1004C000DF93C0E0D0E0BE0185E091E00E94C4016E
:1004D00087E893E10197F1F700C000002196C1156C
:1004E00094E0D90781F72FE78AE196E02150804018
:1004F0009040E1F700C0000060E070E085E091E02E
:10050000DF91CF910C94C401CF93DF93C0E0D0E092
:10051000BE0182E091E00E94C40187E893E1019767
:10052000F1F700C000002196C11594E0D90781F7CA
:100530002FE78AE196E0215080409040E1F700C02B
:10054000000060E070E082E091E0DF91CF910C94D8
:10055000C40160E081E091E00E94F301BC0185E00C
:1005600091E00E94C40161E081E091E00E94F3010A
:10057000BC0182E091E00E94C4018EE091E00E9403
:100580009E01682F8EE091E00E94390188E091E0A1
:100590000E949E01682F8BE091E00E943901D9CF23
:1005A0000E940D020E9436020E945F020E94840295
:1005B0000E94A90288E18093C10086E08093C20076
:1005C0001092C5008FE18093C40008956093C60027
:1005D0008091C00086FFFCCF08958091C00087FF06
:1005E000FCCF8091C60008950E94790080E091E0E0
:1005F0000E94ED0280E091E00E94ED02C82F6FEFB3
:1006000080E091E00E94E6026C2F80E091E00E9481
:10061000E602ECCF81E191E00E94B30042E061E1AB
:1006200071E08EE091E00E94F20043E061E171E050
:100630008BE091E00E94F20045E061E171E088E02A
:1006400091E00E94F20040E061E171E085E091E01C
:100650000E94C10141E061E171E082E091E00C940F
:10066000C101EE0FFF1F0024001C0BBE0790F69186
:08067000E02D0994F894FFCF7E
:00000001FF
